:020000040800F2
:1000000038160020E10100083D0300083D03000808
:100010003D0300083D0300083D0300083D030008C0
:100020003D0300083D0300083D030008E702000807
:100030003D0300083D0300083D0300088F0200084F
:100040003D0300083D0300083D0300083D03000890
:100050003D0300083D0300083D0300083D03000880
:100060003D0300083D0300083D0300083D03000870
:100070003D0300083D0300083D0300083D03000860
:100080003D0300083D0300083D0300083D03000850
:100090003D0300083D0300083D0300083D03000840
:1000A0003D0300083D0300083D0300083D03000830
:1000B0004D210008451C0008A51C00083D03000850
:1000C0003D0300083D0300083D0300083D03000810
:1000D0003D0300082D1F00083D1F00083D030008D8
:1000E0003D0300083D0300083D0300083D030008F0
:1000F0003D03000800F002F800F05EF80AA090E866
:10010000000C82448344AAF10107DA4501D100F0D2
:1001100053F8AFF2090EBAE80F0013F0010F18BF41
:10012000FB1A43F00103184740330000603300001E
:1001300010F8013B0A4413F0030408BF10F8014B08
:100140001D1108BF10F8015B641E05D010F8016B8B
:10015000641E01F8016BF9D1002D15D010F8014B88
:1001600003F00C030C2BA1EB04040ABF10F8013BB5
:10017000A4EB8314A4EB032405F1010314F8016B31
:100180005B1E01F8016BF9D5914238BF10F8013BB5
:10019000D1D370470023002400250026103A28BF41
:1001A00078C1FBD8520728BF30C148BF0B607047E9
:1001B0001FB51FBD10B510BDDFF80CD0FFF7F8FF5D
:1001C00002F083FD03F094F8380E002003B4FFF72B
:1001D000F1FF03BC03F092F802F009B97047000088
:1001E00072B6094880F30988022080F31488BFF3AF
:1001F0006F8FFFF7F1FF0548004770470448054936
:10020000054A064B70470000380E0020F500000834
:10021000380E0020380E002038120020380A002046
:100220002DE9F04FC1F80CD0D0F80CD0BDE8F08F1C
:10023000002383F311882846A04701F06AF900F0F3
:10024000D2FF00DF202080F311883648006810F4C8
:10025000006F02BF002080F311887047EFF3098020
:10026000203880F309884FF08071C1612E498A6976
:100270000968D37F8968926813B1914202D803E07C
:10028000914201D3294900E029498161704710B5A5
:10029000202484F3118801F012F8002080F31188E3
:1002A00084F311881F49096811F4006F04BF80F3BB
:1002B000118810BDEFF30980203880F309884FF0D2
:1002C0008071C16118498A690968D37F8968926819
:1002D00013B1914202D803E0914201D3134900E0E7
:1002E0001349816110BDEFF30980203080F3098844
:1002F000002080F3118870470E4910B50020086077
:10030000091D0D4808601021072000F053F84FF434
:1003100000710A2000F04EF88021BDE810400B204B
:1003200000F048B804ED00E0980100203F0200080A
:100330004302000808ED00E00003FA05FEE70000B4
:10034000254B20F0030C10B463448207D3F800C09F
:10035000D20EFF2494402CEA040C91404CEA010197
:10036000196000F01F020121914042094FF0E02086
:1003700000EB8200C0F88012C0F8001110BC70477A
:100380008107C90E00F01F02012303FA02F243099C
:100390004FF0E02C0CEB8303C3F8802120F0030224
:1003A0000D4810440268FF2303FA01F122EA01011B
:1003B00001607047820720F003030848D20E1844FA
:1003C00003684FF0FF0C0CFA02FC23EA0C03914087
:1003D000194301607047000000E400E018ED00E000
:1003E000202181F31188817F491C8177002181F3CD
:1003F00011887047202181F31188817F4FF000021E
:10040000491E11F0FF01817782F3118806BF017F39
:100410000E297047417F01F0030101290DD0022907
:1004200018BF7047D0E904121161D0E904124A6183
:10043000426C0146104600F0CABAD0E904121161BC
:10044000D0E904124A6100F02EBAF8B51D461646EE
:100450000F46069C00F0E7F9002808BFF8BD2021F0
:1004600081F311882B4632463946009400F07CFF18
:100470000446012060770021204600F020FE002085
:1004800080F311882046F8BDF8B51C4616460F4685
:10049000054600F0C8FA002808BFF8BD202181F306
:1004A0001188009433463A46696800F05DFF0446BF
:1004B0000220607700212046656400F000FE0020E5
:1004C00080F311882046F8BD202383F31188036848
:1004D0000B600160C9488069C1E90102002080F316
:1004E0001188C86070470246202383F3118803688F
:1004F000834209D013688B4202D10868106003E080
:100500001A461B688342F5D1002080F3118870479A
:10051000202181F31188B9498B69996B01EA0002A6
:1005200021EA00009863002080F31188104670478C
:10053000202181F31188B14989698A6B104388634E
:10054000002181F31188704710B5826B11438163DC
:10055000027F082A0DD0092A18BF10BD426A32EA6C
:10056000010118BF10BD00BF00F026FD002141624F
:1005700010BD426A1142F7D110BD2DE9F041046867
:1005800005460E46AC4214BF0027BDE8F081E06886
:100590003043E060D4E90101826B0A438263017F4A
:1005A000082902D0092904D009E0416A0A4206D08C
:1005B00002E0416A914302D100F0FEFC47622468E8
:1005C000AC42E4D1BDE8F081202181F31188C268FA
:1005D000002181F31188C1601046704710B52022B8
:1005E00082F31188826B002411438163027F082A01
:1005F00002D0092A04D00AE0426A114207D003E07F
:10060000426A32EA010102D100F0D6FC446200F0F5
:10061000A4FD84F3118810BD2DE9F0410E46202180
:1006200081F31188046805460027AC421BD0E068BE
:100630003043E060D4E90101826B11438163027FA2
:10064000082A02D0092A04D00AE0426A114207D0DF
:1006500003E0426A32EA010102D100F0ADFC4762D8
:100660002468AC42E3D100F078FD87F31188BDE83F
:10067000F0810022C168C260084670472DE9F04150
:100680000D0006464FF0000414BF0127BDE8F081BD
:1006900007FA04F0284204D0854356F82410204677
:1006A0008847641C002DF3D1BDE8F08170B5054684
:1006B00052488469202080F31188A06B284005D11E
:1006C0000820656200F087FCA06B2840414208408A
:1006D000A16B8143A163002181F3118870BD70B5C6
:1006E000054646488469202080F31188A06B284085
:1006F00005D10820656200F06EFCA06B2840A16B5C
:100700008143A163002181F3118870BD70B5054656
:100710003A488469202080F31188A06B35EA0000F4
:1007200003D00920656200F056FCA06BA843A063CB
:10073000002080F31188284670BD70B505462F480B
:100740008469202080F31188A06B4FF000062840B8
:1007500007D041420840A16B814386F31188A16311
:1007600070BD41B10820656200F077FC0028A4BF8D
:10077000A06B2840EDDA86F31188002070BD70B5BB
:1007800005461E488469202080F31188A06B4FF035
:100790000006284005D0A16B814386F31188A16330
:1007A00070BD41B10820656200F057FC0028A4BF6D
:1007B000A06B2840EFDA86F31188002070BD70B579
:1007C00005460E488469202080F31188A06B4FF005
:1007D000000635EA00000AD029B10920656200F060
:1007E0003CFC002803DA86F31188002070BDA06B62
:1007F000A84386F31188A063284670BD98010020A5
:1008000052485149016000218160C160103000F000
:100810001FB900230360C0E90213083AC1E900329E
:10082000103000F015B92DE9F041050008BF474D23
:10083000C81D20F0070705F1080605F1100000F0BB
:1008400075F93068F8B104464068B84217D307F12B
:10085000080188423CBF2068306009D3E019216854
:1008600040F8081F6168C91B083941603060676043
:10087000256000F089F904F10800BDE8F0812068E6
:1008800026460028DFD100F07FF9296841B107F141
:100890000800884700281CBFE0E80257BDE8F08147
:1008A0000020BDE8F08170B550F8086CA0F1080494
:1008B00006F1080506F1100000F038F928468542D7
:1008C00001D0AC4222D9296809B1A1421ED92160C8
:1008D0002C60616804F108000A182068824205D182
:1008E000426811440831616000682060686805F161
:1008F00008010144A14205D16168084408306860DC
:1009000020682860BDE8704000F03EB92D68D6E749
:1009100070B50E46040008BF0C4C04F1100000F046
:1009200005F90020A168054631B10C4649686D1CE7
:10093000084421680029F8D1002E18BF306000F06B
:1009400023F9284670BD00007F09000878010020C7
:10095000174820F0070117480160174921F00701E7
:10096000416070471349C01D20F00702D1E9000320
:100970001B1A934232BF002002440A6070472021B4
:1009800081F311880B49C01D20F00702D1E9000353
:10099000A3EB000C0023944532BF184602440A60C2
:1009A00083F311887047034841680068081A70474C
:1009B0003F160020000000200040002000230360BC
:1009C000C0E90112704702680A6001607047202286
:1009D00082F3118802680A600160002080F31188A8
:1009E0007047002A1ABF4FF0000C2023704710B444
:1009F00083F3118804680C608CF3118801604468EB
:100A0000521E2144F4D110BC704710B50168002972
:100A10001CBF0A68026004D1826812B14068904726
:100A20000146084610BD10B50146202080F311880C
:100A3000086800281CBF02680A6004D18A68002A7E
:100A40001CBF48689047002181F3118810BD000049
:100A50004060002181600060704770B506468448A0
:100A60008569B06800285CD08168AA68914244D248
:100A70008260017F002938D0042902D005293CD1A9
:100A80001CE0D0E900121160D0E900124A60426A0D
:100A900011460968914204D0D1F808C083686345C3
:100AA000F7D901604B684360486041680860406A5C
:100AB000AA68806881689142DAD31EE0D0E900120A
:100AC0001160D0E900124A60426A114609689142F9
:100AD00004D0D1F808C083686345F7D901604A683B
:100AE000426048604168086007E0D0E90012116088
:100AF000D0E900124A6000F05FFA34462468B4423C
:100B000003D0A168A8688842F8D92C606168696040
:100B10006560696804200D606E62BDE8704000F099
:100B20005ABAB560E86BF060EE6370BD10B5202175
:100B300081F31188FFF791FF002080F3118810BD29
:100B4000816800291CBF0020704749498A6982607A
:100B50008A69D26BC2608969C8630120704720210D
:100B600081F311888168002918BF002008D140490D
:100B70008A6982608A69D26BC2608969C863012010
:100B8000002181F31188704770B5394882692020AF
:100B900080F31188D46B0025E168D1632068A042FE
:100BA00008BFA56017D0106C49B10B688B421CBF01
:100BB0009B68834288BF1846C9680029F5D19060B8
:100BC0002068016821604C60A060C16BE160002179
:100BD000C46300F074FA85F31188204670BD244880
:100BE00010B58369DC6BE168D9632068A04204BF5B
:100BF0000020A06016D01A6C49B1086888421CBF5A
:100C00008068904288BF0246C9680029F5D19A6081
:100C10002068016821604C60A060C16BE160C46322
:100C200000F0CAF9204610BD70B511488469202033
:100C300080F31188E06B0025B8B10146C068E0631D
:100C40000868884208BF8D6008D002680A60516059
:100C50008860C26BCA60C16300F0AEF9E06B002827
:100C6000EBD1206CA06000F078FA85F3118870BD9C
:100C70009801002010B40024DDF804C040604161F8
:100C80008161C0E90241114401610060C0E9073C93
:100C900010BC704770B50446C0686061A061002058
:100CA000A0602068A04214BF6FF0010570BD01680C
:100CB00021604C6000F080F945622068A042F6D1C6
:100CC00070BDD0E9053C8268634504D1002A1CBF91
:100CD0006FF00300704710B5521C82605A1C4261CD
:100CE0001970D0E904128A4224BFC16841610168C9
:100CF000814207D00A6802605060084600F05CF943
:100D000000214162002010BD2DE9F04104460D464E
:100D1000202080F31188E16900291CBF2046884704
:100D20000027A068002808BF9E4E11D129001ED0C0
:100D3000B069446204606368436060604268106048
:100D40000D2000F08AF900280DDBA0680028EDD006
:100D5000401EA060A069411CA161226900788A42FE
:100D60009CBFE168A16187F31188BDE8F0814FF075
:100D7000FF30F8E72DE9F05F04460027D0F81C901B
:100D80001D4692460E46202080F31188DFF814821B
:100D90004FEA070BB9F1000F1CBF2046C847A068F7
:100DA000B8B921466DB1D8F81800416201604A68AF
:100DB000426048604168086029460D2000F04DF906
:100DC00020B18BF311883846BDE8F09FA068002859
:100DD000E7D0401EA060A069411CA161007806F820
:100DE000010B2169A06981429CBFE068A0618BF37F
:100DF00011887F1CBAF1010A1CBF202080F31188E2
:100E0000C8D13846BDE8F09FDDF800C040604161C0
:100E10008161C0E90221114401610060C0E9073C21
:100E2000704770B50446C0686061A0612169081A06
:100E3000A0602068A04214BF6FF0010570BD01687A
:100E400021604C6000F0B8F845622068A042F6D1FD
:100E500070BD2DE9F041044615468846202080F3F8
:100E60001188A0680027002808BF4E4E18D129001D
:100E700010D0B06944620460636843606060426897
:100E800010600D2000F0E9F8002806DA87F31188D9
:100E9000BDE8F0814FF0FF30F8E7A0680028E6D009
:100EA000401EA0606069411C616180F80080D4E947
:100EB000040188429CBFE0686061E16900291CBFB1
:100EC0002046884787F311880020BDE8F081D0E9EB
:100ED00005328168934204D100291CBF6FF00200E3
:100EE000704710B5491C8160511C816114780269FA
:100EF000914224BFC16881610168814207D00A68BC
:100F000002605060084600F057F800214162204618
:100F100010BD2DE9F05F04460027D0F81CA01D4647
:100F200091460E46202080F31188DFF87880BB467A
:100F3000A068B8B921466DB1D8F8180041620160C7
:100F40004A68426048604168086029460D2000F008
:100F500084F820B18BF311883846BDE8F09FA06873
:100F60000028E7D0401EA060606916F8011B421CF3
:100F700062610170D4E9040188429CBFE06860614D
:100F8000BAF1000F1CBF2046D0478BF311887F1C9D
:100F9000B9F101091CBF202080F31188C8D138465F
:100FA000BDE8F09F98010020AF48002140608160BB
:100FB000006040610061704700210177AA498268A2
:100FC00009688B689342FBD201604A6842604860BE
:100FD000416808607047A44B1A4699690877142045
:100FE000C8771068D0F800C0C2F800C0CCF8042060
:100FF000012298610277FFF713B9202181F311884C
:10100000017F4FF0000C002904BF8CF3118870475A
:10101000032904D0052918BF0D290AD103E0416A2C
:101020008A68521C8A60D0E900121160D0E900126F
:101030004A604FF0FF31416280F81CC08A498268E3
:1010400009688B689342FBD201604A68426048603D
:1010500041688CF3118808607047F0B5824C0546F2
:1010600085B0A369481C4FF014074FF0010616D055
:101070007E4A684600F099FAA16922460D77CF773B
:101080001068036813605A60A0610677FFF7C8F81C
:10109000039800281CBF684600F0A3FA0BE0724AD0
:1010A0001D77DF7710681946036813605A60A061E6
:1010B0000677FFF7B5F8A069406A05B0F0BD30B417
:1010C000694C41628368A1690022D1F808C0634578
:1010D0009DBF027764491A460A7784BF624A634615
:1010E0000BD809688B689342FBD201604A68426062
:1010F00048604168086030BC70471268D2F808C088
:101100009C45FAD20A6053684B6051604A6811608E
:101110000122A061027730BCFFF782B8DFF848C136
:101120006046DCF8181002681368036058600120FC
:10113000CCF818201077002008778A68604600688D
:1011400083689342FBD8086042684A6041604868FF
:101150000160DCF81800FFF763B8DFF80CC1DCF8B9
:101160000000DCF8181082688B689A4298BF7047BC
:101170003D4A036813605A600122CCF818000277D8
:101180000020087738488A68006883689342FBD853
:10119000086042684A60416048680160DCF81800F5
:1011A000FFF73EB8DFF8C0C06046DCF818100268F0
:1011B0001368036058600120CCF8182010771420C1
:1011C000C877002008778A68604600688368934281
:1011D000FBD2086043684B60416048680160DCF8FE
:1011E0001800FFF71DB8F0B41F4B00251846996989
:1011F00000680126CA7FD0F800C0C2B11A46C2F802
:1012000000C0CCF80420986106770D7710468A68F4
:101210000068D0F808C09445FAD8086042684A606F
:101220004160486801609869F0BCFEF7F9BF0E4A5A
:101230000C46C2F800C0CCF8042098610677142050
:10124000C8770D7710468A680068D0F808C09445C2
:10125000FAD2086042684A604160486801602146ED
:101260009869F0BCFEF7DCBF98010020FB0F000876
:101270002A4928A089698861FEE708B5FFF73CF88C
:10128000FFF792FE00F088F9FFF762FBFFF7B8FA6C
:101290004021234800F04CF8204988610121017762
:1012A000002181F3118862B61E4A8261AFF23F03CA
:1012B00000910122C0211C4800F07EF808BD70B5E5
:1012C00016488069C17F00291CBF491EC177016A89
:1012D000491C0162154CE068401CE0602068A04297
:1012E00008BF70BD8168491E816006BF00252026A9
:1012F00070BDC168C56002685460026885F31188DA
:1013000022600069884786F3118820688168002977
:10131000EFD070BD69646C6500000000980100208A
:10132000B80100206033000800020020C002002045
:10133000022281600277002242771423C377C0E93A
:101340000F218263026201218177904982610161EC
:101350004A69426148614169086100F1280181627E
:10136000091D0163C162704701442439DDF800C0E2
:10137000C1600B60C168C1F804C0C36884491962C8
:10138000022182600177002141771423C377C0E9ED
:101390000F12816301620122827781617B490161C1
:1013A0004A69426148614169086100F1280181622E
:1013B000091D0163C162704770B504464FF0200CEF
:1013C0008CF31188214424390498E1600B60E168B2
:1013D00000254860E1686E4808620220A26020771C
:1013E00065771420E077C4E90F52A56325620120D8
:1013F000A0776648A56120614169616144616069C7
:101400000021046104F12800A062001D2063E06255
:101410002046FFF754FE85F31188204670BD10B5B5
:101420000146202080F3118858488069046C826846
:10143000A24201D0914200D981600164FFF78DFE84
:10144000002080F31188204610BD10B504462021ED
:1014500081F311880021FFF732FE002181F311880A
:10146000204610BD202181F31188417F41F0040105
:101470004177002080F31188704710B5202282F355
:10148000118801460620FFF7E8FD002080F311884F
:1014900010BD10B5202181F311883E49C968411A59
:1014A0001CBF0620FFF7D9FD002080F3118810BD76
:1014B00010B5202080F3118834480168806989685C
:1014C0008068814228BFFFF76DFE002080F31188FD
:1014D00010BD70B52D498C6904F128056062A06AC1
:1014E000A84207D0A06A0268A262FFF765FDA06A61
:1014F000A842F7D1607F10F0030F05D1D4E90401B1
:101500000861D4E904014161BDE870400E20FFF795
:1015100062BD70B5202181F311881C498C6904F1EA
:1015200028056062A06AA84207D0A06A0268A26289
:10153000FFF742FDA06AA842F7D1607F10F0030FC9
:1015400005D1D4E904010861D4E904014161BDE891
:1015500070400E20FFF73FBD70B50446202080F399
:101560001188207F0E2807D00848A16A8069016091
:10157000A0620720FFF72FFD002080F3118820468E
:10158000656AFEF737FF284670BD0000980100200D
:1015900031020008C002002023484FF0FF314060B4
:1015A000816000210060C1607047DFF87CC0C0E945
:1015B0000323DCF8002093688B4204D21268C91A16
:1015C00093688B42FAD3026053684360506043686B
:1015D00062451860816008BF70479068401A90604B
:1015E0007047114A0168914203D08A6883681A449F
:1015F0008A60D0E900121160D0E900124A6000212F
:10160000C1607047084AD268814207D9824228BF28
:10161000914201D901207047002070478242F9D2DF
:101620008A42F9D2F6E70000C002002000F0A5BD12
:101630000121017000214160704710B5044620204F
:1016400080F311882046616000F09EFD022020702A
:10165000002080F3118810BD10B50446202080F3CF
:101660001188204600F0B9FD01202070002080F391
:10167000118810BD202282F31188C068491E89B2EA
:10168000C162002080F3118870470322027000F0CD
:10169000BDBD10B5202282F311880322027000F034
:1016A000B5FD002080F3118810BD0422027000F007
:1016B000ADBD10B5202282F311880422027000F023
:1016C000A5FD002080F3118810BD0221017000F0FB
:1016D00035BD10B5202181F311880221017000F081
:1016E0002DFD002080F3118810BD10B504460420A4
:1016F0002070204600F09BFD0220207010BD0000ED
:1017000010B500F04BFE00F024F9174800F0A8FDDA
:10171000FFF78CFF00F02CF800F090F8BDE81040C7
:10172000FEF75CBD114A5268814207D9824228BF48
:10173000914201D901207047002070478242F9D2BE
:101740008A42F9D2F6E7094B59680A1858688A4262
:1017500004D9884228BF8242F8D870478842F5D21F
:101760009042F3D3704700000C330008001000E0F3
:1017700000F0C8BA0121017000214160704710B526
:101780000446202080F311886160888820812046EB
:1017900000F0C7FA02202070002080F3118810BDED
:1017A00010B50446202080F31188204600F052FB3B
:1017B00001202070002080F3118810BD202282F3C8
:1017C000118801810069491E89B2C162002080F33D
:1017D0001188704710B5202383F3118800F05EFB59
:1017E000002080F3118810BD10B5202282F31188EB
:1017F00000F072FB002080F3118810BD4FF0FF3322
:101800003030FFF786BB4FF0FF330C30FFF7B2BA32
:101810004FF0FF323030FFF71CBB4FF0FF310C3080
:10182000FFF772BA3030FFF714BB0C30FFF76CBA19
:101830003030FFF76EBB0C30FFF79CBA00F086BB70
:1018400038B5044631482060201D606001202072B8
:1018500015460B46102204F1540104F10C000094CB
:10186000FFF708FA2B46102204F1640104F130005E
:101870000094FFF7C9FA38BD10B50446202080F364
:101880001188204600F074FB02202072002080F3B3
:10189000118810BD10B50446202080F31188204621
:1018A00000F09EFB0120207204F13000FFF7B9FA2E
:1018B00004F10C00FFF7EEF9FFF74FFC002080F376
:1018C000118810BD70B5044640690D4618B9042151
:1018D000201DFEF752FE294604F10C00FFF7F1F936
:1018E0000028A8BF70BD8021201DBDE87040FEF714
:1018F00044BE70B504463030FFF7E9FA051E03DA3E
:101900000821201DFEF739FE284670BD78330008F7
:101910001B49496881607047194949688268891A7A
:10192000184A1268891A8160C268914284BFC160F6
:1019300070470269914288BF1146016170471249A0
:1019400001601249416000218160C160491E01614E
:10195000704710B50B4C86B000200B4920600091F9
:101960000A49CDE901100390401E04906846FFF734
:10197000CFFF0199684688470298206006B010BDE5
:10198000001000E0080000201119000819190008D3
:101990000FB42DE9F04F83B007460EAD4FF02D097F
:1019A0000D9810F8011B0D90002902BF03B0BDE88F
:1019B000F00F5DF814FB252904D03868826838469A
:1019C0009047EDE701786C4626464FF0000C2D2934
:1019D00003D1401C4FF0010C0D9001784FF020080E
:1019E0002E2903D1401C4FF030080D904FF0000B12
:1019F0000D9911F8010B0D91A0F13001092998BF43
:101A0000C8B207D92A2803D000212E2807D012E017
:101A100015F8040B0BEB8B0100EB410BE8E70D9A7B
:101A200012F8010B0D92A0F13002092A98BFD0B232
:101A30000ED92A280AD06C2818BF4C280DD0A0F146
:101A40004102192A94BF0123002310E015F8040B6A
:101A500001EB810100EB4101E1E7DDF834A0012356
:101A60009AF800201AB110460AF101020D9264287A
:101A700039D00EDC552874D006DC442818BF49281C
:101A800031D04F286FD010E0582868D063280CD18F
:101A90000DE0732812D004DA692824D06F2804D10D
:101AA00061E075285DD0782859D0207004E015F8E1
:101AB000040B4FF020082070641C87E055F8046B7D
:101AC0004FF02008002E08BF5CA6002908BF47F68B
:101AD000FF7134462078002878D0491E0029A8BF1D
:101AE000641CF7DA72E055F8042B002A02DA04F8D5
:101AF000019B52420A21134604F10B0A1046B2FB25
:101B0000F1F201FB120030303928C8BFC01D0AF8BD
:101B1000010DB3FBF1F3002BF0D1A4EB0A0000F1AF
:101B20000B03012BD8BF0123AAF10101601E13F0A2
:101B3000010F03D011F8012F00F8012F5A1009D01E
:101B400091F801A080F801A011F802AF00F802AFEF
:101B5000521EF5D11C4439E003E004E0FFE71022F7
:101B600002E00A2200E0082255F8040B04F10B03FE
:101B7000014600BFB0FBF2FA02FB1A0030303928F0
:101B8000C8BFC01D03F8010DB1FBF2F1504600299A
:101B9000F0D1E01A00F10B0ABAF1010FD8BF4FF0F3
:101BA000010A591E601E1AF0010F03D011F8012F0F
:101BB00000F8012F5FEA6A0207D04B78437011F8F2
:101BC000023F00F8023F521EF7D15444A4EB060A2C
:101BD000ABEB0A04002CB8BF0024BCF1000F08BF17
:101BE0006442002C13DA31782D2908BFB8F1300F88
:101BF00006D13868761C826838469047AAF1010AF7
:101C000038684146826838469047641CF8D1BAF17A
:101C1000010A08D4386816F8011B826838469047D4
:101C2000BAF1010AF6D5002C3FF4BAAE3868414645
:101C3000826838469047641EF8D1B1E6286E756C0C
:101C40006C29000070B5AD4C2069018A828902EAD6
:101C50000105E943018215F0020F03D060680169B4
:101C60002046884715F0040F03D06068816920463C
:101C7000884715F0080F03D06068016A204688473E
:101C800015F0100F03D06068816A2046884715F070
:101C9000010F03D06068816820468847BDE8704026
:101CA000FEF7D0BA70B5964C2069018A828902EAA3
:101CB0000105E943018215F0020F03D06068016954
:101CC0002046884715F0040F03D0606881692046DC
:101CD000884715F0080F03D06068016A20468847DE
:101CE00015F0100F03D06068816A2046884715F010
:101CF000010F03D06068816820468847BDE87040C6
:101D0000FEF7A0BA10B57D48FFF734FD7B497D484A
:101D1000086101F11400FFF72DFD79497A48086147
:101D200010BD2DE9F04104460078002501282CD093
:101D300020690580206985812069058220694563C5
:101D4000206985632069C56320690564206945624F
:101D50006168E0680968B0FBF1F02169401E088500
:101D600020892169401E80B2C86260682169808D27
:101D70008880616800200A7B02F00F02012A2FD0C0
:101D8000022A08BF02202BD02CE05C485F4E604F37
:101D9000A0420DD1F06940F00200F061306940F0DE
:101DA00002003061356170211D20FEF7C9FAE7603D
:101DB0005348A0420DD1F06940F00400F061306951
:101DC00040F004003061356170211E20FEF7B8FA42
:101DD000E760216946F66800088321698883B7E7D0
:101DE00040F001000A7D02F00F02012A04D0022A0D
:101DF00008BF40F0200001D140F010000A7F02F03F
:101E00000F02012A04D0022A08BF40F4007001D159
:101E100040F4807091F8241001F00F01012904D0E2
:101E2000022908BF40F4005001D140F480502169DC
:101E3000088421690120888260688068002818BFB2
:101E40000120216988812069058221698520088017
:101E5000BDE8F08170B504460078022818BF70BD57
:101E6000002021690880216988812169088223482E
:101E7000264DA04206D11D20FEF782FAE86920F027
:101E80000200E8611E48A04218BF70BD1E20FEF788
:101E900077FAE86920F00400E86170BD4FF0340C77
:101EA00003690CEB810C43F80C201023426803EB10
:101EB000C103D258002A08BF704703699A894FF0BE
:101EC000020C0CFA01F1114218BF70470A439A81C3
:101ED0000069C943018270474FF0340C03690CEB71
:101EE000810C002243F80C2000698289022303FA46
:101EF00001F122EA0101818170470000D002002037
:101F0000E4020020000400400008004000100240ED
:101F100000A24A047E48018841F080010180704798
:101F20007C48018841F080010180704710B57A48F3
:101F300000F075F8BDE81040FEF784B910B5774899
:101F400000F06DF8BDE81040FEF77CB910B5744A9A
:101F500000217148FFF774FC6F497248724A486764
:101F600000216E48FFF76CFC6C497048486710BD53
:101F700070B50C00054608BF6D4C287A012816D1B3
:101F800065486C4EA84207D1B06940F48040B0610A
:101F9000C0212520FEF7D4F96048A84207D1F06996
:101FA00040F40030F061C0212620FEF7C9F95D4AF7
:101FB00061492268686FB1FBF2F10181E18841F06B
:101FC00040010182218941F001018182A18842F210
:101FD0002C1211438181002101800188808870BD0D
:101FE000017A022918BF70470022416F8A810A8254
:101FF0008A82494A4F49824206D1886920F480404A
:1020000088612520FEF7BCB9444A824218BF704758
:10201000C86920F40030C8612620FEF7B1B92DE967
:10202000F047456F0646B5F80C902C88B5F804A02B
:1020300014F00F0F4FF020074FF000081AD00021C6
:1020400014F0080F18BF802114F0010F18BF41F0E1
:10205000200114F0020F18BF41F0400114F0040FEA
:1020600018BF41F4807187F31188301DFEF785FA9F
:1020700088F3118814F4807F0CD087F311884FF413
:102080000071301DFEF779FA88F31188288820F452
:102090008070288014F0200F08D087F311880AF090
:1020A000FF013046FFF70EFC88F3118819F0800F0E
:1020B00018BF14F0800F14D087F3118806F1300098
:1020C000FEF705FF0028A8BFA88008DA0821301D08
:1020D000FEF753FA29F0800040F04000A88188F311
:1020E000118814F0400F08BFBDE8F08787F311880E
:1020F0001021301DFEF741FA88F3118829F04000C5
:10210000A881288820F040002880BDE8F0870000E2
:102110000C3801400C440040F802002070030020FD
:10212000151F000800380140211F0008004400402E
:10213000983300080010024000512502C2680021B7
:102140001180C2681182C06881817047414810B512
:10215000C268002111820278042A07D1022202708B
:10216000C2681180C2681182C26891814168496861
:102170008847BDE81040FEF765B836494FF080400B
:10218000C8600846FFF754BA70B5044600780025C9
:10219000012804BF2F48A0420FD12F48C16941F048
:1021A0000101C161016941F0010101610561702115
:1021B0001C20FEF7C5F82948A060D4E90110096881
:1021C000B0FBF1F0E168401E0D80E26808219180CB
:1021D000E1680885E068858170BD0178022918BF33
:1021E00070470021C2681180C2689181C268118263
:1021F0001849814218BF704710B51C20FEF7C0F87F
:102200001548C16921F00101C16110BDC268491EB4
:10221000D162C26801219182C36800225A62C368F8
:102220001A82C2689181C068052101807047C26826
:10223000491ED162C26801219182C26800211182C7
:10224000C2680D211180C068018A11F0010FFBD016
:1022500070470000E80300200010024000A24A047A
:1022600040498A6940F2FD131A438A613E4A016877
:1022700011603E4A81681160121F416811603C4A3A
:10228000C16811603B4A41691160121F0169116008
:1022900039498269CA60026A4A60C2690A60374A7B
:1022A000416A1160364AC16A1160121F816A116069
:1022B000344A016B1160344A816B1160121F416B0B
:1022C0001160324AC16B1160314A416C1160121FBA
:1022D000016C11602F49826CCA60026D4A60C06C4B
:1022E00008607047F0B4032A08BF016102D0042AD5
:1022F00008BF4161284B9D5C00221446134694465A
:1023000004261B01120124014FEA0C1C11F0800F5E
:102310000CBF43F00F032A4311F4004F0CBF4CF0E5
:102320000F0C2C4349001B01120124014FEA0C1C25
:1023300011F0800F0CBF43F00F032A4311F4004F3C
:102340000CBF4CF00F0C2C434900761ED9D14168CC
:1023500001EA0C0121434160016819401143016009
:10236000F0BC7047001002400C0801400408014016
:102370000C0C0140040C0140001001400C14014001
:10238000041401400C180140041801400C1C0140C9
:10239000041C014000200140A433000831480169B9
:1023A0004FF0FF32026100210161C368C260C16069
:1023B0004FF0E0222C4B53619161072111612B49B1
:1023C0000A6842F080720A6029490A6842F00102F4
:1023D0000A60C16941F08051C161C16941F0006189
:1023E000C1612448016841F48071016070471D4853
:1023F000016841F001010160016811F0020FFBD09A
:10240000016801F0F901016000214160416811F0AB
:102410000C0FFBD1016841F480310160016811F4B7
:10242000003FFBD0416841F4E8114160016841F090
:1024300080710160016811F0007FFBD00E4941609E
:102440000E4A12211160416841F002014160416869
:1024500001F00C010829FAD1016821F001010160A5
:1024600070470000001002403F190100FCED00E041
:10247000001000E00070004000641D0000200240D9
:1024800070B5202080F31188FD4D0024286820B10C
:1024900032214162FEF790FD2C6084F3118870BDFB
:1024A000FA49FB4DF7A089694FF480742E1F8861AB
:1024B0002C604FF4FA70FEF7E0FF34604FF4FA70CE
:1024C000FEF7DBFFF4E782B0DFF8C0A34FF4FA7049
:1024D00000900025DAF81810EEA0DFF8B493DFF8CA
:1024E000C4B32F462E4601244FF02008C1F818002F
:1024F00088F31188E249DAF8180008600220FEF734
:102500006AFDDAF818000021406A81F31188012879
:1025100011D0022815D032283BD0012FE8D1012E4E
:10252000E6D80226072D80F05D81DFE805F0355DF5
:1025300097C0E8F9F8000127701CC6B200253C4698
:10254000EDE74FF48060C9F800004000C9F80000D2
:102550004000C9F800004000C9F800001020CBF886
:1025600000004020CBF80000CBF800808020CBF8A2
:102570000000012F08D0CCA1D248FFF709FA0027AC
:102580003E463D460124B3E7CFA1CE48FFF700FA0F
:10259000F5E7012FACD1C4E7012C20D0502CA7D8EF
:1025A000D148C4F150030068D0A100F00102C54831
:1025B000FFF7EEF9DA494FF480600860D94910203E
:1025C0000860D9480099FFF774F8601C84B2512C58
:1025D0008ED1D6A1BB48FFF7DBF901253CE0D4A1A1
:1025E000B848FFF7D5F9DBE7CF480099FFF761F866
:1025F000BD48006810F0010F06D0D3A1B148FFF725
:10260000C7F90124022573E7A02C06D8DAA1AD484A
:10261000FFF7BEF9601C84B26AE74FF48060C9F826
:1026200000004000C9F800004000C9F80000400068
:10263000C9F800001020CBF800004020CBF80000C3
:10264000CBF800808020CBF80000D3A19D48FFF795
:102650009FF900273E463D46012449E7502C3FF6AE
:1026600047AF4FF48060C9F800001020CBF800009D
:10267000C101AB480160AB48C0F800809A48C4F182
:1026800050030068CB4900F001028E48FFF780F943
:10269000A5480099FFF70DF8601C84B2512C7FF417
:1026A00027AFA2A18748FFF773F90325D4E7102CC1
:1026B0003FF61EAF4FF40060C9F80000CBF8008071
:1026C0004100974801609749402008608648C4F15E
:1026D00010030068B8A1C0F340027A48FFF758F928
:1026E00091480099FEF7E5FF601C84B2112C7FF43D
:1026F000FFAE8EA17348FFF74BF90425ACE78A487B
:102700000099FEF7D6FF7848006810F0020F08D055
:10271000B5A16C48FFF73CF901240525E8E652E035
:1027200028E0A02C06D8BBA16648FFF731F9601C51
:1027300084B2DDE64FF48060C9F800004000C9F8BB
:1027400000004000C9F800004000C9F80000102057
:10275000CBF800004020CBF80000CBF800808020B0
:10276000CBF80000B2A15748FFF712F900273E4608
:102770003D4671E7A02C3FF6BBAE4FF48050C9F840
:1027800000004020CBF800006549C00108606549A1
:10279000802008605448C4F1A0030068AAA1C0F3D7
:1027A00040024848FFF7F4F85F480099FEF781FFC0
:1027B000601C84B2A12C7FF49BAE5CA14148FFF762
:1027C000E7F8062548E74FF40050C9F800008020DC
:1027D000CBF80000A9A13B48FFF7DAF800273E46F6
:1027E0003D4685E6ABA13748FFF7D2F880E627499A
:1027F000ADF5167DA9A08969AB4DAC4CC1F81800A8
:102800004FF47A70FEF739FE4FF0FF334FF4FA724F
:10281000694604F10C00FEF7ADFAA5A1684600F088
:102820006BFC070000F0CC81A3A100F065FC002840
:1028300025D0C01BC6B2642E88BF642632463946F6
:102840007DA800F09DFC31467DA800F0E9FB4FF02B
:10285000FF330B2299A104F13000FEF75AFB4FF031
:10286000FF330D2205F1080104F13000FEF751FBA2
:102870004FF0FF3302222DA104F1300024E184E166
:102880000C000020626C696E6B657200980100207C
:10289000140C01404F6470616C5F766C616B6E6FFD
:1028A00000000000100801404F6470616C206E65EC
:1028B00062796C20616B7469766F76616E2E0D0A99
:1028C00000000000F80200200D0A4F6470616C20C7
:1028D0007A727573656E20757A69766174656C6558
:1028E0006D2E0D0A000000000808014028312F3429
:1028F00029094F7465766972616E692076696B612A
:102900002E2E2E20537472656368613A2025642C44
:10291000205A627976613A20253364200D00000048
:10292000100C014014080140E80300200D0A0000CB
:102930005679706F757374656E69207A6168616A23
:10294000656E6F210D0A0000537472656368612023
:102950006F74657672656E612E20506F6B72616365
:102960006F76616E692076206E61706F7573746525
:102970006E692E0D0A00000043656B616E69206E62
:1029800061206F74657672656E6920737472656319
:1029900068792E0D000000000D0A4E656C7A6520E6
:1029A0006F74657672697420737472656368752ECE
:1029B0000D0A0000CC33000828332F342909507247
:1029C0006570616C6F76616E69206C6973752E2E0F
:1029D0002E204C69733A2025642C205A6279766146
:1029E0003A202533640D00004C69732073746C61C8
:1029F00063656E2E20506F6B7261636F76616E69D6
:102A00002076207072657461766F76616E692E0D26
:102A10000A00000043656B616E69206E612073746B
:102A20006C6163656E69206C6973752E0D00000022
:102A30000D0A4E656C7A6520737075737469742025
:102A40006C69732E0D0A000028342F3429095A614D
:102A50007461766F76616E692062616C6F6E752E3F
:102A60002E2E204C69733A2025642C205A627976E8
:102A7000613A20253364200D000000005679706F04
:102A8000757374656E6920756B6F6E63656E6F210B
:102A90000D0A00004E4943210D0A00004750535FC4
:102AA0004E4D454100000000080A00207003002040
:102AB00024475047474100002A0000004C617469D8
:102AC000747564653A200000FEF723FA4FF0FF3377
:102AD0000C22F7A104F13000FEF71BFA4FF0FF3390
:102AE0000E2205F1150104F13000FEF712FA4FF045
:102AF000FF330222AFF2CC1104F13000FEF709FAE5
:102B00004FF0FF330B22EDA104F13000FEF701FA84
:102B10004FF0FF330A2205F1230104F13000FEF7E4
:102B2000F8F94FF0FF330222AFF2002104F1300038
:102B3000FEF7EFF94FF0FF330922E3A104F1300073
:102B4000FEF7E7F94FF0FF330122E91D04F13000F1
:102B5000FEF7DFF94FF0FF330222AFF2302104F12C
:102B60003000FEF7D6F94FF0FF3332467DA904F16D
:102B70003000FEF7CEF94FF0FF330222AFF25421BE
:102B800004F13000FEF7C5F93AE64FF0FF330222B8
:102B9000AFF2682104F13000FEF7BBF94FF0FF33CC
:102BA0002A22CCA104F13000FEF7B3F94FF0FF3335
:102BB0004FF4FA72694604F13000FEF7AAF91FE6F5
:102BC0004FF0FF332122CEA104F13000FEF7A1F92E
:102BD00016E6F0B595B00746D2A100F0FDFA202622
:102BE000D24C002518B3D2A1384600F0F5FA0028DF
:102BF0002AD0D1A1384600F0EFFAD14C78B3D1A158
:102C0000384600F0E9FA58B35422D049684600F03B
:102C100085FA6B1E5322694604F13000FEF779F9FC
:102C2000CB48016881F08001016015B0F0BD86F3EA
:102C30001188206820B101214162FEF7BDF92560AD
:102C400085F3118815B0F0BD86F31188206800283F
:102C5000F6D002214162FEF7AFF92560F0E700E00F
:102C60000BE015B004F13000BDE8F0404FF0FF3349
:102C700040F26712B749FEF74CB9B7A1B048FEF76A
:102C800087FEBA4C206810F0010F04D0B8A1AC4800
:102C9000FEF77EFE03E0B9A1A948FEF779FEBAA1CE
:102CA000A748FEF775FE206810F0020F06D015B099
:102CB000B8A1BDE8F040A248FEF76ABE15B0B8A1C1
:102CC000BDE8F0409E48FEF763BEA0B00025FEF7C9
:102CD00017FDFEF7D2FA00219948FEF7CDFDB34C5F
:102CE00011224FF400712046FFF7FCFAB049B148B9
:102CF000FEF7C2FD102204212046FFF7F3FAAE4E84
:102D0000062280213046FFF7EDFA062221153046D3
:102D1000FFF7E8FA2015A94C206041000622304652
:102D2000FFF7E0FAE0142060410006223046FFF78A
:102D3000D9FAA0142060410006223046FFF7D2FAEB
:102D4000601420609E4810210160402101604FF016
:102D50002008C0F80080802101609A499A48FEF757
:102D60006CFC0024994B40224FF4987198480094D1
:102D7000FEF722FB974B40224FF46C71964800946B
:102D8000FEF71AFB954B40224FF49871944800943B
:102D9000FEF712FB6A4F631E40F267126D4907F19E
:102DA0003000FEF7B6F8614E4FF0010B4FF0020A0B
:102DB0004FF0FF33012201A907F10C00FDF7DAFF04
:102DC0009DF804000D2801D00A2D6ED30DF11809CD
:102DD000002554A1484600F0FFF910B354A148461D
:102DE00000F0FAF938B354A1484600F0F5F970B391
:102DF00054A1484600F0F0F950B3542253490AA8B0
:102E000000F08CF96B1E53220AA907F13000FEF77F
:102E100080F84F48016881F0800101608DF818400A
:102E2000C6E788F31188306870B1C0F824B0FEF7A7
:102E3000C3F8346008E088F31188306820B1C0F826
:102E400024A0FEF7B9F8346084F31188E6E700E0C7
:102E500009E04FF0FF3340F267123E4907F13000BE
:102E6000FEF757F8DAE73CA13548FEF791FDDFF8A9
:102E7000FC90D9F8000010F0010F04D03CA13048BC
:102E8000FEF786FD03E03DA12D48FEF781FD3EA142
:102E90002B48FEF77DFDD9F8000010F0020F05D099
:102EA0003CA12748FEF774FDB8E7A1E09AE00000D6
:102EB0004C6F6E6769747564653A2000416C746983
:102EC000747564653A2000005374617475733A2018
:102ED000000000004E656E616C657A656E20756B52
:102EE0006F6E636F76616369207A6E616B204E4D01
:102EF0004541207A7072617679202A0D0A0000001F
:102F00004E656E616C657A656E207A616361746589
:102F10006B204750474741207A70726176790D0ADD
:102F2000000000006F6470616C0000000C00002065
:102F30007A7275730000000068656C700000000014
:102F4000F8020020636865636B0000001434000819
:102F50000C0C0140100000200D0A537461762073A0
:102F60007472656368793A20000000000808014027
:102F70004F74657672656E610D0A00005A61767253
:102F8000656E610D0A00000053746176206C6973F0
:102F9000753A2000416B7469766E690D0A00000075
:102FA000526F7A65706E7574790D0A0000080140E1
:102FB000C033000870030020000C0140140C0140D5
:102FC00010080140B8330008E8030020A1240008DD
:102FD000F8030020EF27000858060020C724000847
:102FE00028050020AFF248010C48FEF7D1FC15E798
:102FF000732806D006A94A1954704855681CC5B2F2
:10300000D6E688F31188306820B1C0F824A0FDF717
:10301000D3FF346084F31188CAE60000F802002070
:103020002DE9F00300231D461E469C461A46002942
:1030300084BF00272F4C47D8BDE8F0037047012A12
:1030400004D0022A18BF032A09D014E010F8038024
:1030500004F80C800CF1010C0CF0FF0C34E004EBD4
:10306000060810F803C088F808C006F1010C0CF03F
:10307000FF064FF0000C042A18BF052A07D104EB05
:10308000050910F803806D1C89F81580EDB2062A39
:1030900002D0092A18D10FE004EB0C08254408F8E7
:1030A000017C04EB060888F807702F75C51815F821
:1030B000015CE571002507E004EB050910F80380C9
:1030C0006D1C89F82380EDB210F80380B8F12C0F45
:1030D00004BF521CD2B2092A05D9601980F82270A7
:1030E000BDE8F00370475B1CDBB29942A7D8BDE88E
:1030F000F0037047080A002030B505460B462A4603
:1031000013F8014B12F8010B08B1A042F8D01CB122
:10311000002802D06D1CF1E7284630BD10B5203ADA
:10312000C0F00B80B1E81850203AA0E81850B1E880
:103130001850A0E81850BFF4F5AF5FEA027C24BF36
:10314000B1E81850A0E8185044BF18C918C0BDE82D
:1031500010405FEA827C24BF51F8043B40F8043BF6
:1031600008BF7047D20728BF31F8023B48BF11F8AB
:10317000012B28BF20F8023B48BF00F8012B704705
:1031800010B5044610F0030F08BF11F0030F40F014
:1031900015804FF0013E121FC0F20E8051F8043B23
:1031A000A3EB0E0C2CEA030C1CEACE1C08BF40F863
:1031B000043BF0D0A1F1040102F10402521E08DB2D
:1031C00011F8013B002B00F8013BF7D1114600F04C
:1031D00046F8204610BD00004FF0013C50F8042B8B
:1031E00051F8043B9A4221D1A2EB0C03934313EA1A
:1031F000CC1317D150F8042B51F8043B9A4215D147
:10320000A2EB0C03934313EACC130BD150F8042B1D
:1032100051F8043B9A4209D1A2EB0C03934313EA01
:10322000CC13DBD04FF00000704700BFD01A01BABA
:10323000B1FA81F101F0180122FA01F0CB40C1F19D
:103240002001DBB2C0B2C01A2CFA01F3D11A9143AB
:1032500011EAC311E6D170477047704770474FF0CD
:1032600000020429C0F0128010F0030C00F01B8053
:10327000CCF1040CBCF1020F18BF00F8012BA8BF61
:1032800020F8022BA1EB0C0100F00DB85FEAC17C25
:1032900024BF00F8012B00F8012B48BF00F8012BD8
:1032A00070474FF0000200B5134694469646203909
:1032B00022BFA0E80C50A0E80C50B1F12001BFF4EF
:1032C000F7AF090728BFA0E80C5048BF0CC05DF855
:1032D00004EB890028BF40F8042B08BF704748BFA3
:1032E00020F8022B11F0804F18BF00F8012B704717
:1032F0000446AFF300802046FCF768FF0149182020
:10330000ABBEFEE72600020070470000FDFFFFFF96
:10331000844B333388488488FFFFFFFF8888443814
:1033200083AA8888FFFFFFFF88888888BBBB8B88BB
:10333000FFFFFFFF448B888888888888FFFFFFFF96
:10334000888888888888888800000000000000003D
:10335000000000000000000000000000000000006D
:103360006D61696E00164211040448080C101418AF
:10337000001C1D1E1F200000FD1700080718000874
:10338000111800081B180008251800082B18000841
:1033900031180008371800088025000000000040A0
:1033A00000000000040204080800030708080808D9
:1033B000080808080B0F0000E8030000812400083B
:1033C00080250000000000400000000028322F345B
:1033D000290956656E74696C206F74657672656E26
:1033E000202D3E206E6166756B6F76616E6920627E
:1033F000616C6F6E752E2E2E20537472656368613A
:103400003A2025642C205A627976613A202533646B
:103410000D0000004E65706C61746E7920707269E9
:103420006B617A210D0A093C6F6470616C3E2070FB
:10343000726F207A6168616A656E692073656B7668
:10344000656E63650A0D093C7A7275733E20707271
:103450006F207A727573656E69207679706F7573F7
:1034600074656E690A0D00008834000800000020B1
:10347000780100003001000868350008780100205C
:10348000C014000094010008D2000100072F0D0AAB
:103490000D0A2A200270570D0A5669746120766160
:1034A00073204175746F6D617469636B792056790F
:1034B000706F7573746563204D6574656F62616CC0
:1034C0006F6E7520312E310D0A5A61706F6A656E0C
:1034D00069207679766F64753A0D0A094750494F2D
:1034E000423130202D20737472656368611412318B
:1034F00014700776656E74696C1312322770046C51
:1035000069731012332310057A61746127400569CD
:103510002F6F645D200A0D0A5072696B617A795FC2
:10352000123C161004616C3E263368617A100473F5
:10353000656B2E1363658341A7100B6E690A0D0935
:103540003C7A727573261106419FA11C10086865AC
:103550006C703E206EBC040535766564612B0005F9
:08356000000D0A00000000004C
:04000005080000F5FA
:00000001FF
